:0300000002036593
:0C036500787FE4F6D8FD75815502035442
:10000300000000002E2A3A0088F8000000000000DB
:10001300000088FF000000C020C0008088FF0000AF
:1000230000010201000088FF000000000000000042
:1000330088FF000808002E2A3A00080F0800000075
:1000430000000400000000000200000000000100A6
:1000530000000000008000000000004000000000DD
:100063000020000000000010000000000008000055
:100073000000000400000000000200000000000176
:1000830000000000000080000000000040000000AD
:100093000000200000000000100000000000080025
:1000A3000000000004000000000002000000000047
:1000B300010000000000008000000000004000007C
:1000C30000000020000000000010000000000008F5
:1000D3000000000000040000000000020000000017
:1000E300000100000000000080000000000040004C
:1000F30000000000200000000000100000000000CD
:1001030008000000000004000000000002000000DE
:10011300000001000000000000800000000000401B
:10012300000000000020000000000010000000009C
:020133000008C2
:10035400C29475903E51E77139512151A851CA8018
:01036400FA9E
:1001D200E4FBFAC293EF70047D0D80027D0FE4FC14
:1001E200C292ED30E304D2918002C291D292ED2507
:1001F200E0FD0CBC04EAD291C292E4FCEB25E0FBE8
:10020200EA33FAD292C2923091054303018003533A
:0E02120003FE0CBC0CE6D293EA540FFEAF03C1
:0102200022BB
:1002A800E4F551E4FF31D2AB07AA067C007D673143
:1002B8004774082551F8A6070551E551C3944940EC
:0102C800E253
:0102C9002212
:1002CA00E4F55174082551F8E6FFE551240AFD5179
:0C02DA00690551C3E551648094C940E7F8
:0102E60022F5
:020269008D52B4
:10026B00755305EF3395E0FE7C007D0631358E54DA
:10027B008F55AD53AF527171743F2555F582740094
:10028B003554F583E493FF71030555E5557002056D
:0C029B00541553C3E5536480948050D682
:0102A7002234
:10022100E4F551F552AD52AF517171E4F553E55218
:1002310075F00AA4F554AF54EF3395E0FE74032F23
:10024100F58274003EF583E493FF71030553055471
:10025100C3E5536480948A40DDE4F5510552D3E54A
:07026100526480948540BE49
:010268002273
:10030300D295E4FEEF30E704D2968002C296D297EC
:0A031300C297EF25E0FF0EBE08EAD6
:01031D0022BD
:10031E00C295E4FEEF30E704D2968002C296D297E1
:0A032E00C297EF25E0FF0EBE08EABB
:0103380022A2
:1002E700C294D2947F21711E7FBC711E7F07711E3D
:0C02F7007F13711E7F20711E7F0C611EA2
:10033900E4FDFC7F80711E7F40711EE4FF71030D97
:0A034900BD00010CBC01F4BDF8F189
:010353002287
:0C037100EF2480FF711EED2440FF611E90
:10013500EF8DF0A4A8F0CF8CF0A428CE8DF0A42EDE
:02014500FE2298
:10014700C2D5EC30E709B2D5E4C39DFDE49CFCEED3
:1001570030E715B2D5E4C39FFFE49EFE12017DC3CD
:10016700E49DFDE49CFC800312017D30D507C3E4C8
:060177009FFFE49EFE2242
:10017D00BC000BBE0029EF8DF084FFADF022E4CC66
:10018D00F875F008EF2FFFEE33FEEC33FCEE9DEC2F
:10019D00984005FCEE9DFE0FD5F0E9E4CEFD22ED75
:1001AD00F8F5F0EE8420D21CFEADF075F008EF2FBF
:1001BD00FFED33FD4007985006D5F0F222C398FDB0
:0501CD000FD5F0EA224D
:00000001FF
